:020000001828BE
:080008009000900E030E910020
:10001000040E92000A0E93000B1D10280B1178217C
:10002000130E8A00120E8400110E8300100E0900B8
:100030008316C030810083120B08DF398B00A301C7
:10004000A201A401A5010030A8002208A9000030E7
:10005000AA0012210130A8002408A9000130AA003A
:1000600012210230A8002508A9000030AA001221A0
:100070000130A8002408A9000130AA001221023092
:10008000A8002508A9000030AA001221831605083F
:1000900010388500831205081039A70027080F3C87
:1000A000013003180301FF390130031D0030003C0B
:1000B000031D5B2838280030A8002208A900003062
:1000C000AA0012210130A8002408A9000130AA00CA
:1000D00012210230A8002508A9000030AA00122130
:1000E0008316050810388500831205081039A7000B
:1000F0000F302702013003180301FF390130031DBF
:100100000030003C031D85285B2883160108F83960
:100110000438810083120B08DF39A0388B000030CF
:10012000A8002208A9000030AA0012210130A8006E
:100130002408A9000130AA0012210230A8002508D5
:10014000A9000030AA001221831605081038850086
:10015000831205081039A70027080F3C0130031847
:100160000301FF390130031D0030003C031DB92895
:100170008F280030A8002208A9000030AA00122110
:100180000130A8002408A9000130AA001221023081
:10019000A8002508A9000030AA001221831605082E
:1001A00010388500831205081039A7000F30270288
:1001B000013003180301FF390130031D0030003CFA
:1001C000031DE328B9280B08DF398B000030A80095
:1001D0002208A9000030AA0012210130A80024083A
:1001E000A9000130AA0012210230A8002508A900A8
:1001F0000030AA00122183160508103885008312EA
:1002000005081039A70027080F3C01300318030127
:10021000FF390130031D0030003C031D1029E62882
:100220001C281129083094000430950002309600F3
:1002300001309700C0309800F9309900A4309A003E
:10024000B0309B0099309C0092309D0082309E001F
:10025000F8309F008030A0009830A10008308D0059
:100260008E0129088F0003108F1B03148E0D0A3096
:100270008E0203183D298E0703108F0D8D0B332935
:100280000E08183E84000008AB0000302802013040
:10029000031C0301FF39031956292808033C0130C8
:1002A000031C0301FF39031956290130003C0319CF
:1002B000772983160508F03985000608003986007D
:1002C00083120508F03985002A08003C03196A29C1
:1002D0007F30AB05060800392B0486000508F0398D
:1002E0008D002808143E840000080D0485000800D5
:1002F0008C012308013E03188C0AA3000A30230254
:10030000031C8429A301852108008C012208013ED9
:1003100003188C0AA2000A302202031CA529A2019C
:100320008C012408013E03188C0AA4000A30240220
:10033000031CA529A4018C012508013E03188C0A81
:0C034000A5000A3025020318A5010800E2
:00000001FF
